:0200000480007A
:100000006F004005732F2034930F8000630AFF03B5
:10001000930F90006306FF03930FB0006302FF038A
:10002000170F0000130F4F2463040F0067000F0029
:10003000732F203463540F006F00400093E19153FD
:10004000171F000023203FFC171F0000232E0FFA6C
:100050006FF01FFF930000001301000093010000E8
:10006000130200009302000013030000930300003A
:100070001304000093040000130500009305000022
:10008000130600009306000013070000930700000A
:1000900013080000930800001309000093090000F2
:1000A000130A0000930A0000130B0000930B0000DA
:1000B000130C0000930C0000130D0000930D0000C2
:1000C000130E0000930E0000130F0000930F0000AA
:1000D000732540F16310050097020000938202012E
:1000E000739052307350447497020000938202015F
:1000F00073905230735000189702000093824202AE
:10010000739052309B021000939252039382F2FF3D
:100110007390023B9302F0017390023A73504030A7
:100120009702000093824201739052307350203046
:100130007350303093010000970200009382C2ECAC
:1001400073905230130510001315F501635C050020
:100150000F00F00F930110009308D0051305000065
:100160007300000093020000638A02007390521033
:10017000B7B200009B82921073902230735000300F
:10018000372500001B05058073200530970200000D
:100190009382420173901234732540F17300203032
:1001A00093012000B70703049B87172097200000C6
:1001B000938040E503A70000B70303049B8313204B
:1001C000631A770693013000B70704059B87273031
:1001D00097200000938000E303A71000B7030405F5
:1001E0009B8323306318770493014000B70705060B
:1001F0009B873740972000009380C0E003A7200032
:10020000B70305069B8333406316770293015000C2
:10021000B70706079B87475097200000938080DE32
:1002200003A73000B70306079B834350631477008E
:10023000631030020F00F00F6380010093911100F2
:1002400093E111009308D0051385010073000000AD
:100250000F00F00F930110009308D0051305000064
:10026000730000009302400073232034E39462FC87
:1002700013870700F32210349382420073901234E4
:1002800073002030731000C0000000000000000068
:10029000000000000000000000000000000000005E
:1002A000000000000000000000000000000000004E
:1002B000000000000000000000000000000000003E
:1010000000000000000000000000000000000000E0
:1010100000000000000000000000000000000000D0
:1010200000000000000000000000000000000000C0
:1010300000000000000000000000000000000000B0
:081040000000000000000000A8
:1020000001020304050607080000000000000000AC
:040000058000000077
:00000001FF
